:100000003BC0A0C154C053C052C051C050C04FC02B
:100010004EC04DC04CC04BC04AC049C048C047C08C
:1000200046C045C044C00902120001010080190900
:10003000040000000000000012011001FF00000891
:10004000C016DC050401010200010E035500530037
:1000500042006100730070001C0377007700770096
:100060002E00660069007300630068006C002E00BB
:10007000640065000403090411241FBECFE5D4E029
:10008000DEBFCDBF10E0A0E6B0E0E2E9F1E102C0E2
:1000900005900D92A236B107D9F710E0A2E6B0E0C4
:1000A00001C01D92AC3AB107E1F760D870C8A8CF83
:1000B000CF93DF9360918800635067FD13C08091F8
:1000C0008500CCE0D0E0C81BD109C457DF4F809138
:1000D00084008D3209F457C08091620087FD9BC077
:1000E000109288008091600084FF40C060916100A0
:1000F0006F3F09F43BC0693008F46FC068506093EB
:1001000061008091780098E889278093780068E002
:100110008091620087FD1DC040918600509187004C
:1001200086FF70C0FA01862FA9E7B0E094919D93F5
:1001300031968150D9F7262F215030E02F5F3F4F65
:10014000240F351F3093870020938600C62FCC5F85
:100150004FC089E790E0D3D6682F893008F4A1C05A
:100160008FEF80936100CEE1C093600094E186B38D
:10017000837031F49150D9F7109289001092830066
:10018000DF91CF910895683009F0AACF83EC809376
:1001900078008AE580936000109262008881807602
:1001A00009F043C09A81109281008981811147C072
:1001B0001092820021E830E082E0309387002093A3
:1001C00086008F3FA9F19F81911104C09E819817ED
:1001D00008F4892F8093610083CF10926100809191
:1001E000780098E8892780937800611191CFC4E066
:1001F00089E790E0A3D0CC3009F4B6CF8FEF80939D
:100200006100B2CFDA01862FE9E7F0E09D9191938A
:100210008150E1F790CFCE01DFD68F3FF1F08823F8
:1002200009F45ECF109261005BCFCE01C3D4C9CF79
:10023000988197FD16C090E890936200CBCF8530EF
:1002400091F0863001F18830D1F0893091F021E8C9
:1002500030E08A3021F180E0B0CF8EE18093600001
:100260003FCF8E81E8CF9093890021E830E080E095
:10027000A4CF90938B0021E830E080E09ECF2BE864
:1002800030E081E09ACF8B81813001F18230B1F092
:10029000833051F080E090E49093620092CF81E04F
:1002A0008CCFC82FCC5FA4CF911118C084E790E009
:1002B000909387008093860084E0EDCF86E290E003
:1002C000909387008093860082E1E5CF88E390E0F9
:1002D000909387008093860082E1DDCF913051F0CA
:1002E0009230C1F68AE490E0909387008093860074
:1002F0008EE0D1CF88E590E09093870080938600D0
:100300008CE1C9CF85B7836085BF8BB780648BBF15
:100310000895A82FB92F80E090E041E050EA609561
:1003200030E009C02D9182279795879510F084279A
:100330009527305EC8F36F5FA8F30895EADF8D93C9
:100340009D930895CF93CFB7CF93DF93C395B09B81
:10035000E9F7B09B0BC0B09B09C0B09B07C0B09B36
:1003600005C0B09B03C0B09B01C089C06F93C09112
:100370008500DD27C457DF4F2F9365E5B09B03C091
:100380002F916F91E6CF0F931F934F9320E040E1A1
:100390005F9306B3037000FB27F93F9350E03BE007
:1003A00039C0137040642F77012F5F5F1EC0406813
:1003B00016B313702F7752501FC0406406B32F77C7
:1003C0000370D1F15F5F00C023C0406216B32F7786
:1003D000137091F15F5F00C025C00370102751506A
:1003E00012F45D5F0000115027952C3F16B3C8F63C
:1003F00013700127015027952C3FC8F642274993D7
:1004000006B3037010274F73115027952C3FA8F6A1
:100410004695469516B3137079F00127015027953C
:100420002C3F98F66B5A60F3315006B3B0F600C01B
:1004300010E41ABF002717C03B503195C31BD040B2
:1004400010E41ABF0881033CF9F00B34E9F0209165
:1004500083001981110F1213EDCF093651F10D32BE
:1004600011F0013E39F700938A003F915F914F915F
:100470001F910F912F916F91CAB7C6FD67CFDF9182
:10048000CF91CFBFCF91189520918A00222369F395
:1004900010918800112339F534303AF130938800F7
:1004A00020938400109185003BE0311B3093850040
:1004B0001CC0009188000130B4F40AE5309160005E
:1004C00034FD14C000936000C8E7D0E013C00527D6
:1004D00010E000C0000008BB1AC0052710E0221F72
:1004E0001DC010E021C04AE502C032ED432FC4E137
:1004F000D0E032E017B31360C09A08B317BB53E0E3
:1005000020E865E320FF052708BB279517951C3FCA
:10051000F0F66695B8F7B1F720FF052708BB2795D9
:1005200017951C3FD0F62795179517FF0527000054
:100530001C3F08BBB0F629913A9519F70C7F109132
:100540008900110FC651D04008BB11F010938300F1
:1005500010E41ABF016017B31C7F402F4C7F54E09A
:100560005A95F1F708BB17BB48BB7FCF682F58E0FF
:1005700080E07091A8002091A70067FD1EC0C3987D
:10058000660F880FB4998F5FC59A32B7472F4150D5
:1005900030F092B7931B9217E0F34150D0F7C59813
:1005A00032B7472F415030F092B7931B9217E0F3C8
:1005B0004150D0F7515009F70895C39AE1CF8FB950
:1005C000779BFECF8FB1089521E19695879577951A
:1005D00067952A95D1F72091A6002617D9F0609348
:1005E000A600E091A300F091A4008DE40995E091AC
:1005F000A300F091A40080E00995E091A300F091A0
:10060000A4008091A6000995E091A300F091A400B8
:1006100080E0099408958091A5008DB98091A20091
:100620008EB908958823B1F0893008F04AC026EBCE
:1006300032E03093A4002093A30091E09093A800AF
:10064000853001F1C0F08730A1F168F588E0809332
:10065000A70008958FED92E09093A4008093A300EB
:100660001092A20081E08093A7008093A80082E509
:100670008093A5000895833001F140F080E28093DB
:10068000A700089580E18093A7000895823039F093
:1006900080E88093A70082E08093A800089580E816
:1006A0008093A7000895883099F782E08093A7008F
:1006B000089584E08093A700089580E48093A700C4
:1006C00008952FED32E03093A4002093A300109200
:1006D000A20091E09093A7009093A800893049F080
:1006E00030F28B3051F08C3011F681E58093A5000B
:1006F000089583E58093A500089582E58093A50081
:100700009093A200089522B73091A8009091A7007D
:10071000315030F082B7821B8917E0F33150D0F7A7
:10072000089587B38C6287BBC298C59822B7309171
:10073000A800432F9091A700415030F082B7821B50
:100740008917E0F34150D0F7C29A22B7315030F008
:1007500082B7821B8917E0F33150D0F7C29880919D
:10076000A3009091A4008F5D924019F01092A60012
:1007700008958091A5008DB98091A2008EB9109244
:10078000A600089587B3837D87BB88B3837D88BB2C
:100790001DB80895CF93DF93C0E2E091A300F091DC
:1007A000A4008CEA0995E091A300F091A40083E5F0
:1007B0000995E091A300F091A40080E00995D82F5D
:1007C000E091A300F091A40080E00995D33509F4ED
:1007D0003AC01DB822B73091A800432F9091A700CE
:1007E000415030F082B7821B8917E0F34150D0F7B7
:1007F000C29A22B7432F415030F082B7821B89172B
:10080000E0F34150D0F7C29822B7315030F082B7B0
:10081000821B8917E0F33150D0F7E091A300F091EB
:10082000A40082E0EF3DF80739F0C15009F0B9CFDC
:1008300081E0DF91CF9108958091A5008DB98091DD
:10084000A2008EB9F2CF80E0DF91CF910895CF92D0
:10085000DF92EF92FF926B017C01B6DED701C601F9
:1008600081709927AA27BB27880F880F880FE091EE
:10087000A300F091A40080620995D701C60139E078
:10088000B695A795979587953A95D1F7E091A300EE
:10089000F091A4000995D701C601B695A795979543
:1008A0008795E091A300F091A4000995E091A30041
:1008B000F091A40080E0FF90EF90DF90CF9009943A
:1008C000CF92DF92EF92FF920F931F93CF93DF931C
:1008D0006B017C01C42FD22F77DE97018601017056
:1008E000112722273327802F880F880F880FE09148
:1008F000A300F091A40080640995D701C60159E0D6
:10090000B695A795979587955A95D1F7E091A3004D
:10091000F091A4000995D701C601B695A7959795C2
:100920008795E091A300F091A4000995E091A300C0
:10093000F091A4008C2F0995DD23A9F0CF3789F021
:10094000D2B7CEE1C701B60182DF8F3761F482B73B
:100950008D1B813510F0D2B7C150C111F3CF81E0AA
:1009600003C08FE0B2D080E0DF91CF911F910F9153
:10097000FF90EF90DF90CF900895CF92DF92EF92AB
:10098000FF920F931F93CF93DF931F92CDB7DEB7E4
:100990006B017C01498318DEE091A300F091A40073
:1009A0008CE40995D701C60179E0B695A79597958E
:1009B00087957A95D1F7E091A300F091A40009956D
:1009C000D701C601B695A79597958795E091A300A5
:1009D000F091A4000995E091A300F091A40080E0BB
:1009E000099549814F3FE1F002B71EE1C701B60109
:1009F0002EDF8F3F99F482B7801B813510F002B74C
:100A000011501111F3CF81E00F90DF91CF911F9121
:100A10000F91FF90EF90DF90CF90089580E0F4CF9A
:100A20008FE053D080E0F0CF1F93CF93DF931F92DE
:100A3000CDB7DEB7182FE091A300F091A40080EAB3
:100A400099830995E091A300F091A4009981892FE1
:100A50000995E091A300F091A400812F0995E09100
:100A6000A300F091A40080E00F90DF91CF911F913F
:100A700009941F93CF93DF9300D0CDB7DEB7182F23
:100A8000E091A300F091A40080EC6A83998309951A
:100A9000E091A300F091A4009981892F0995E0913C
:100AA000A300F091A400812F0995E091A300F0919B
:100AB000A4006A81862F09958EE107D080E00F900F
:100AC0000F90DF91CF911F910895882349F030E076
:100AD00022B792B7921B9035E0F33F5F3813F8CFFF
:100AE0000895BD9ABB98C39A50E217D05A95E9F77A
:100AF0000895AC0188E605D0842F03D089E601D0A3
:100B0000852F0FD028E030E0382780FB869506D06F
:100B10002A95D1F730FB02D000D06894BB98C39AD5
:100B200016F0C398BB9AE091AA00F091AB00319700
:100B3000F0F7C59AE6B3E3FBE091AA00F091AB00B1
:100B40003197F0F7C598089520ECE7DF46F42A9531
:100B5000E1F780E02AE1E5DF2A95E9F7DECF28E03A
:100B600030E0DBDF869587F938272A95D1F7D5DF86
:100B700027F9322772F3D1DFD0CFDB01742FB9DF31
:100B800084E2BFDFE1DF8D937A95D1F70895DB0131
:100B9000742FAFDF83EFB5DF8DE1B3DF84E6B1DF24
:100BA0008D91AFDF82E7ADDFCFDF8078D9F77A951F
:100BB00089F70895CF93DF93EC018981813089F122
:100BC000823009F4A8C0833009F45FC08430A1F1F9
:100BD000873009F47FC0853009F4FEC0863009F4FF
:100BE0009EC0883009F4D1C0893009F4FAC08A3037
:100BF00009F425C18B3009F451C18C3009F461C16D
:100C00008D3009F473C18E3009F475C18F3009F449
:100C1000F9C0803109F41AC18F3709F434C180E07A
:100C20002BC09A9B54C080916300FCDC109264003E
:100C3000A99877DD80E020C080916400811110C008
:100C40005B8140E08A81482B662757FD6095762FAF
:100C500040936D0050936E0060936F00709370002E
:100C60009F8180E02E81822B90937200809371008F
:100C700082E0809373008FEF25E630E030938700A9
:100C800020938600DF91CF910895E091A300F09129
:100C9000A4008A81099580936500E091A300F091FA
:100CA000A4008B81099580936600E091A300F091E8
:100CB000A4008C81099580936700E091A300F091D6
:100CC000A4008D8109958093680084E0D5CF85E0EC
:100CD000A9DCACCF80916400811110C05B8140E041
:100CE0008A81482B662757FD6095762F40936D00CB
:100CF00050936E0060936F00709370009F8180E04E
:100D00002E81822B909372008093710083E08093F8
:100D100073008FEFB1CF36DDA99A80E0ADCF80911F
:100D20006400811110C09B8180E02A81822BAA2758
:100D300097FDA095BA2F80936D0090936E00A093BD
:100D40006F00B09370003C812D81822F8F70809353
:100D50007600822F807F40E1849FC0011124830FA1
:100D6000911D909375008093740020FD809377000F
:100D70009F8180E02E81822B90937200809371007E
:100D800081E0809373008FEF77CF809164008111B1
:100D900010C09B8180E02A81822BAA2797FDA09515
:100DA000BA2F80936D0090936E00A0936F00B09364
:100DB00070001092750010927400109276009F815E
:100DC00080E02E81822B909372008093710084E0EA
:100DD000809373008FEF50CFDDDC8093650081E05E
:100DE0004BCF81E0809364008A819B81AC81BD817F
:100DF00080936D0090936E00A0936F00B09370008D
:100E000080E03ACF9B8180E02A81822BAA2797FD40
:100E1000A095BA2F80936D0090936E00A0936F0001
:100E2000B09370009F8180E02E81822B909372009E
:100E30008093710085E0809373008FEF1DCF8A81CE
:100E4000809363001092650081E016CF9B8180E063
:100E50002A81822BAA2797FDA095BA2F80936D0037
:100E600090936E00A0936F00B09370009F8180E01C
:100E70002E81822B909372008093710086E0809384
:100E800073008FEFF9CE81E08093650010926600C9
:100E9000109267001092680084E0EECE9B8180E0A3
:100EA0002A81822B9093AB008093AA00C29ABA9AAF
:100EB00083E00BDEC298A99880E107DE12DE80E0B5
:100EC000DBCE80EC1EDE80E01CDE8AE0FEDDC29A16
:100ED00085E0FBDDC29885E0F8DD87B3837D87BBC5
:100EE00088B3837D88BBA99A80E0C6CE2DDE80932F
:100EF000650081E0C1CE8A8104DE80E0BDCE0F9323
:100F00001F93CF93DF93582F792F062F20917300D3
:100F1000322F3250323050F0253009F441C00FEFFB
:100F2000802FDF91CF911F910F910895662381F15A
:100F300080916D0090916E00A0916F00B091700053
:100F4000C52FD72F10E01BC06FDD888380916D0007
:100F500090916E00A0916F00B09170000196A11D5C
:100F6000B11D80936D0090936E00A0936F00B093BD
:100F700070001F5F2196101749F0209173002230F6
:100F800019F7BC01CD0163DC8883E0CF083040F65F
:100F900010927300802FDF91CF911F910F910895D0
:100FA000462F682F80916D0090916E00E6DD809154
:100FB0006D0090916E00A0916F00B0917000800F55
:100FC000911DA11DB11D80936D0090936E00A093A3
:100FD0006F00B0937000A4CFFF920F931F93CF9335
:100FE000DF93382F792F162F20917300213071F065
:100FF000243061F0263009F48BC0FF24FA948F2D41
:10100000DF91CF911F910F91FF900895112309F463
:10101000ABC080916D0090916E00A0916F00B09177
:101020007000C32FD72F00E0F12C4EC02091740028
:1010300030917500232B09F050C021E04881BC019C
:10104000CD013EDC209171003091720021503109B8
:101050003093720020937100232BE1F410927300FF
:101060008091760081FF36C02091770030E080913A
:101070007400909175002817390761F160916D0037
:1010800070916E0080916F0090917000488175DCC6
:10109000FF24F39480916D0090916E00A0916F00F9
:1010A000B09170000196A11DB11D80936D009093C9
:1010B0006E00A0936F00B09370000F5F2196011730
:1010C00009F49DCF20917300213009F4AFCF6881DE
:1010D000D0DCB8CFFF24F394DDCF20E04881BC0101
:1010E000CD01EEDB809177008150809377008111F4
:1010F000A9CF60916D0070916E0080916F0090910A
:10110000700048813ADC80917400809377009ACF18
:10111000462F682F80916D0090916E0038DD809190
:101120006D0090916E00A0916F00B0917000810FE2
:10113000911DA11DB11D80936D0090936E00A09331
:101140006F00B09370008091710090917200811BCC
:1011500091099093720080937100892B29F4109269
:101160007300FF24F3944BCFF12C49CF12BA18BA75
:101170008BEF81BB8FEF87BB17BA83E084BB9EEFF9
:1011800095BB83BFBFD8789493D792D7FDCFF894FF
:02119000FFCF8F
:021192005AFF02
:00000001FF
